:1000000083160030850086008312023085000030A0
:10001000850005309E000310013086003B20860DD0
:100020003B20061F0F280514000005109E0B0B280F
:1000300005309E007F30860000009D0B1C280514B3
:10004000000005109E0B1A289A0B182860309000AB
:100050009100100892001108930086170000920B7F
:100060002E2886130000930B3228940B2928900326
:10007000910B2928002801309A009B0B3D289C0BEE
:080080003D289A0B3D28080001
:00000001FF
